:1078000011241FBE8DEF9AE09EBF8DBF04B714BE3A
:1078100088E18093600010926000409100085091D0
:1078200001086F917F9199C00F928F939F931F9240
:107830000FB60F9211244F936F938091DA0080FF5F
:107840003FC02BC00F920FB68F939F93EF93FF9380
:1078500088278093850080938400EEE7F1E0908193
:107860008917980B919309F45D9890818917980B6B
:10787000908309F428987C9B05C05BD319F0C10163
:1078800001961C01FF91EF915CC080E189BD82E10E
:1078900089BD09B400FEFDCF08958091D80080FF16
:1078A0000FC08091DA008E7F8093DA008091D9003A
:1078B00080FF04C0EADF81E08EBB02C019BC1EBAA3
:1078C0008091E10080FF0BC0BBD180FF08C0BBD11D
:1078D0008091D800806275D219BC85E08EBB809102
:1078E000E10084FF1AC0ACD184FF17C0CEDF8091C5
:1078F000D8008F7D66D28FEE2AD0A2D18F7E816094
:10790000A5D180918501882331F48091E30087FD22
:1079100002C081E001C084E08EBB8091E10083FF62
:107920000CC08ED183FF09C087EF11D082E08EBBDF
:10793000109285010BD087D19BD16F914F910F9001
:107940001F909F918F910FBE0F9018958EEF009012
:10795000E10008220092E100089510BA80E181BBA5
:10796000579A5F98A0E0B1E0E0E7FFE705900D923D
:10797000AD37E1F71D92BB30E9F75F9A01FD0FC00B
:1079800000FF03C07C9B0BC008C003FF08C0675703
:10799000774729F04757574711F0CBD251F4E3D13D
:1079A00078942224332439D0B4D2C10180549F4129
:1079B000D0F3F89481E08093E00010926F00109271
:1079C0008100109285001092840081E085BF15BE71
:1079D0005D9828980C9400002ED107C0DBD002C01F
:1079E00095D239F02AD182FFFBCF85FFF7CF809166
:1079F000F1000895082E83E01FD185FD07C014D142
:107A000002C084D249F019D180FFFBCF0092F1006F
:107A10005D9A84E680937E0108950DD182FFD5C0E2
:107A2000289A84E680937F01D7DF182FF2018534EE
:107A300031F48CE49DE11C0182D28DE096C0843546
:107A400011F4CADFFACF8C34C1F38035B1F3843737
:107A500021F484E4CFDF80E088C0813611F489E529
:107A600084C0813431F4B8DFF82FB6DFE82F7CD240
:107A7000E4CF803711F483E578C0833539F4C0E072
:107A8000D1E08991B7DFC730E1F770C0863521F4C6
:107A900081E3B0DF82E369C0833731F487E8AADF8E
:107AA00085E9A8DF8EE161C0853639F4E0E8F7E7C3
:107AB00084D0E058F040E0F7C0CF823631F489E559
:107AC00099DF80E097DF80E850C0823419F0873674
:107AD00009F037C0222433247FDFD82F7DDFC82F61
:107AE0007BDF082F8554823008F03EC010926F0073
:107AF000173659F406C0063411F4859101C027D217
:107B000079DF2197C2F72F0118C04F01063461F4C5
:107B100054D00AC061DF063431F4C0FB16F0182ED1
:107B200046D0082E01C017D22197A2F72F010634A4
:107B300011F4F4013AD08DE05DDF82E080936F00B4
:107B400015C08237E1E049F08634E0E031F08E3450
:107B5000E3E019F0813531F4E2E0F0E089E087BF3D
:107B6000849103C08B3111F08FE344DF83E0DED1D9
:107B70005BD095FF03C009C0C9D139F15ED080FF49
:107B8000FBCF52D002C0C2D101F157D080FFFBCF52
:107B900084E0CCD18BE749C010D090E40D901D90CB
:107BA00006D09A95D9F7E058F04085E007C081E00B
:107BB00087BFE89511243296089583E001D081E1D2
:107BC00087BFE89507B600FCFDCF089590918D0121
:107BD00080918E01913231F0913A61F5813251F507
:107BE00038D083C0803231F534D090D1E9F085307F
:107BF000D9F023D083FD18C082FFF7CF04C0F7DE91
:107C00008193615031F09091F3008091F200892BC3
:107C1000B1F7C0DF611549F704C078D129F085308C
:107C200019F00BD080FFF9CF8EE79091E8008923FF
:107C30008093E800089584E079D18091E800089568
:107C40008091E2000895FCDF8E7F80618093E200E6
:107C500008955AD1E6E8F1E067E0089582E061EC2A
:107C600009D083E061E802D084E060E842E103C02B
:107C700080E060E042E05AD181E007D01092ED0050
:107C80006093EC004093ED0008959091EB00892BF8
:107C90008093EB00089560E0923039F0933041F02A
:107CA000913079F4E7E062E10CC0E9E16EE309C0EC
:107CB000813018F4E7E564E004C019F4EBE562E212
:107CC00000C0F1E0089580918D0188234CF402C03A
:107CD0001DD151F0B2DF82FFFBCF5CCF17D121F075
:107CE000ACDF80FFFBCFA0DF08954091930150915E
:107CF00094014617510510F490E028C0611511F069
:107D0000462FFACF91DF40E0F7CF00D159F185300F
:107D100049F193DF83FD3ECF90DF82FD20C080FFDD
:107D200015C03091F3002091F20005C0819180933D
:107D3000F10041502F5F411519F028303105B0F3A3
:107D400050E02830310509F451E06EDF4115E9F6C5
:107D50005523D9F604C0DAD029F0853019F06DDF4B
:107D600082FFF9CF17CF20E82093610010926100C5
:107D700081E085BF32E035BF209A2898559A5D98FA
:107D8000109289008AEF8093880030936F0083E01F
:107D90008093810081E08093D7008AE482BF1092B3
:107DA000D8001092E2001092DA001092E10080E810
:107DB00008D019BC1EBA1092E0005ADF89E046DFF5
:107DC00081E98093D8000895EDE8F1E010DE819319
:107DD000E539E1F7FBDE31DF83FF91C080918D0152
:107DE00090918E01913009F170F09330F1F095305F
:107DF00009F444C0963009F456C0983009F460C0C4
:107E0000993059F767C0823841F7809191018DD040
:107E10002091EB001092E90077D0229526952170F1
:107E20002093F1001092F10052C0882311F08230AB
:107E3000A1F68F71823089F680918F018823D1F469
:107E400020919101277049F22093E9008091EB0085
:107E500080FF10C0933011F480E20BC080E115DF89
:107E600081E0880F2A95E9F78093EA001092EA00F2
:107E700088E00BDF1092E90047D02AC0882391F4F4
:107E800010918F0110680FB7F8943ED01CDFD5DE3B
:107E900080FFFDCF1093E300103883E009F482E007
:107EA0008EBB0FBF2CC08058823048F580918F0167
:107EB00090919001F0DE603011F126D016DF1FC0E6
:107EC0008038E9F421D0809185018093F100ACDE07
:107ED000FADE15C0882399F490918F01923078F4DE
:107EE0009093850111D0EFDE80918501882321F4E4
:107EF0008091E30091E087FD94E09EBBAFDE9DDEC4
:107F000083FF089580E2C1DE87EF8FCE8EB3882392
:107F10000895FCDF69F08091E9008F931092E900E9
:107F20008CDE83FF01C050DF8F9187708093E90062
:107F30000895E0E0F0E08591949101960895F201B2
:107F4000F695E795F999FECFF2BDE1BD0895F7DF0B
:107F5000F89A80B508C0F3DF1FBA80BD0FB6F89459
:107F6000FA9AF99A0FBE3196EE0FFF1F2F0108956E
:107F700041524455424F591201100102000008417C
:107F800023370001000001000109023E0002010048
:107F900080320904000001020201000524001001E2
:107FA000042402040524060001070582030800FFDB
:107FB00009040100020A0000000705040210000184
:107FC0000705830210000104030904220341007223
:107FD000006400750069006E006F0020004D0069AC
:0E7FE00000630072006F0020002000200000EF
:047FFC00CDCDFBDC10
:040000030000780081
:00000001FF
